:10000000830100308A00C028FC0003088301C3007C
:100010000A08C4008A017008C7000B1D10281128A7
:100020001628013083120313A9070B11831203133F
:100030000C1C1B281C28B528C203C208031D21283C
:1000400022283F280108A8070318A90A01308506BD
:100050003030C2002808A6002908A700851C3128D6
:100060003228352814309500392864308312031360
:10007000950083120313A801A90181010B11FE3021
:10008000831203138F00BB308E008601A10A063055
:100090002102031C4C284D284E28A1018312031372
:1000A00085150000851181288312031305150000B2
:1000B00005112C08A3009728831203132D08A30011
:1000C0009728831203132A08A300A308031D692895
:1000D0006A286C281530A3009728831203132B0875
:1000E000A3009728831203132E08A30097288312D6
:1000F00003132F08A300972883120313A301972843
:100100009728831203132108003A03195428013A4F
:1001100003195C28033A03196128013A03196D2871
:10012000073A03197228013A031977287C2804300A
:1001300083120313210203189E289F28AE2816302D
:100140002302031CA428A528A628A30101308A00A5
:1001500083120313230800218600B228831203139D
:1001600023088600831203130C100313831247081D
:10017000F00044088A0043088300FC0E7C0E09004E
:10018000213084004230D620203084002130D62017
:1001900083010730C600FF30C50042308400433081
:1001A000DA208301402C04068001840A0406031D22
:1001B000D3280034F000E6208000840A040870068A
:1001C00003190034DB2883120313C500C61BF12872
:1001D000461BF92846088A004508C50A0319C60ABD
:1001E00082008313461883174508C50A8400000857
:0201F000080005
:1001FA00031383120800820777340634B334973422
:10020A00C634D534F5340734F734D734E734F43404
:10021A007134B634F134E134E6347034C3348034A2
:10022A0010340034F0000030711870070310F00D1C
:0C023A000310F10CF10803190800192949
:1005400083120313B1003108F0000310F00C031004
:10055000F00C0310700CB000B008031DB02AB12AD3
:10056000B22ABA2A83120313B003B008031DB92AB2
:10057000BA2AB22A03138312080083120313B001AC
:10058000B100C72AF63083120313B107B00A0A304C
:100590008312031331020318CE2ACF2AC22A8312F0
:1005A0000313300884008313310880003008D82AF0
:1005B00003138312080083120313BF00C100BF0896
:1005C000031DE32AE42AE52AFF2A9F30831203133E
:1005D000C000C008031DED2AEE2AEF2AF72A831275
:1005E0000313C003C008031DF62AF72AEF2A83125B
:1005F0000313BF03BF08031DFE2AFF2AE52A0313C6
:1006000083120800831203138501860107309F00BF
:10061000F330831685008601E830810020308B009E
:10062000313083129000FE308F00BB308E000C10F2
:1006300083160C140B178312051564308316920071
:1006400064308312950097017C3092000C30970043
:100650008B1703138312080083120313B8011030A1
:10066000B9000E30BA001130BB001130BC00BD0122
:100670001530BE001030AA000E30AB001130AC00B7
:100680001130AD00AE01AF018B170730B700B71FB7
:100690004A2B4B2B4C2B3D2C00308312031327028B
:1006A000653003192602031C562B572B582B3D2C63
:1006B00006308312031338020318672B5F2B3808A8
:1006C000393E840083130008682B1530682B652B96
:1006D00083120313AA003808F000F1010130F0077B
:1006E0000318F10A7108803AF20080307202063075
:1006F000031970020318852B7D2B380A393E8400BC
:1007000083130008862B1530862B832B831203134B
:10071000AB003808F000F1010230F0070318F10ACD
:100720007108803AF20080307202063003197002BC
:100730000318A42B9B2B3808023E393E84008313F8
:100740000008A52B1530A52BA22B83120313AC0098
:100750003808F000F1010330F0070318F10A7108BE
:10076000803AF200803072020630031970020318DA
:10077000C32BBA2B3808033E393E8400831300088C
:10078000C42B1530C42BC12B83120313AD00B80A40
:1007900002303802031CCD2BCE2BCF2BB801831295
:1007A0000313AE01AE0AAF01831203132E082E0706
:1007B000AE002E08083A031DDE2BDF2BE12B103094
:1007C000AE000A30DB22AE08031DE72BE82BD42B4A
:1007D00083120313AE01AF01AF0A0A30DB2283128A
:1007E00003132F082F07AF002F08083A031DF92B1A
:1007F000FA2BFC2B1030AF000A30DB22AF08031DB0
:10080000022C032CEF2B803083120313AF00031054
:10081000831203132F0CAF002F08083A031D112C6D
:10082000122C142C0430AF000A30DB22AF08031D59
:100830001A2C1B2C072C803083120313AE00AF013F
:100840000A30DB220310831203132E0CAE002E0895
:10085000083A031D2C2C2D2C2F2C0430AE000A300E
:10086000DB22AE08031D352C362C222C83120313F9
:10087000B703B71F3C2C3D2C4C2B031383120800ED
:1008800083120313B001B101B201B301B401022319
:100890002C23B301B4018B13831203132608B10078
:1008A0002708B2008B176430F4000030F5000030E8
:1008B000F6000030F7003208F1003108F000F201D4
:1008C000F301C2270C30F4000030F5000030F600D0
:1008D0000030F7001E277008B1007108B200273001
:1008E0003202103003193102031C772C782C7C2C37
:1008F0000F30B1002730B2008312031334083202E4
:10090000031D842C33083102031C872C882C8F2C68
:100910003108B3003208B400C830B0009C2C8312F8
:100920000313B0080319952C962C982CB0039C2C1B
:1009300083120313B301B401E830F2000330F30073
:10094000831203133208F1003108F000E426740822
:10095000AA00E830F2000330F3003208F100310859
:10096000F000E4267008B5007108B6006430F200AB
:100970000030F3003608F1003508F000E426740872
:10098000AB006430F2000030F3003608F1003508A7
:10099000F000E4267008B5007108B6000530320298
:1009A000DD3003193102031CD62CD72CE82C323051
:1009B000F2000030F3003608F1003508F000E426BC
:1009C0007408F0000530F10070081721AC00FA2C13
:1009D0003230F2000030F300831203133608F100C6
:1009E0003508F000E4267408F0000530F1007008C6
:1009F0001721AC0083120313AD0101303202903095
:100A000003193102031C052D062D082D2E140B2D64
:100A1000831203132E10033083120313320220308B
:100A200003193102031C152D272D03303402203009
:100A300003193302031C262D1D2D04303402B0305F
:100A4000031933020318262D252D272D282D2A2D95
:100A5000292D2C2DAE142F2D83120313AE1004302C
:100A6000831203133202B03003193102031C392DF3
:100A70004B2D04303402B03003193302031C4A2DCD
:100A8000412D0630340240300319330203184A2D39
:100A9000492D4B2D4C2D4E2D4D2D502D2E15532DBA
:100AA000831203132E1106308312031332024030D7
:100AB00003193102031C5D2D6F2D063034024030C6
:100AC00003193302031C6E2D652D07303402D0301C
:100AD0000319330203186E2D6D2D6F2D702D722D9D
:100AE000712D742D2E16772D831203132E120730BD
:100AF000831203133202D03003193102031C812DFB
:100B0000932D07303402D03003193302031C922D89
:100B1000892D093034026030031933020318922DF5
:100B2000912D932D942D962D952D982DAE169B2DB0
:100B300083120313AE1209308312031332026030A2
:100B400003193102031CA52DB72D09303402603082
:100B500003193302031CB62DAD2D0A303402F030D8
:100B6000031933020318B62DB52DB72DB82DBA2DA4
:100B7000B92DBC2D2E17BF2D831203132E130A304F
:100B8000831203133202F03003193102031CC92D02
:100B9000DB2D0A303402F03003193302031CDA2D46
:100BA000D12D0C3034028030031933020318DA2DB2
:100BB000D92DDB2DDC2DDE2DDD2DE02DAE17E32D27
:100BC00083120313AE130C308312031332028030EE
:100BD00003193102031CED2DFF2D0C30340280303F
:100BE00003193302031CFE2DF52D0E303402103094
:100BF000031933020318FE2DFD2DFF2D002E022EAA
:100C0000012E042E2F14072E831203132F100E30E3
:100C1000831203133202103003193102031C112E08
:100C2000232E0E303402103003193302031C222EFF
:100C3000192E0F303402A030031933020318222E6C
:100C4000212E232E242E262E252E282EAF142B2E99
:100C500083120313AF100F30831203133202A0303C
:100C600003193102031C352E472E0F303402A030F9
:100C700003193302031C462E3D2E1130340230304E
:100C8000031933020318462E452E472E482E4A2EAE
:100C9000492E4C2E2F154F2E831203132F11113076
:100CA000831203133202303003193102031C592E10
:100CB0006B2E11303402303003193302031C6A2EBC
:100CC000612E12303402C0300319330203186A2E29
:100CD000692E6B2E6C2E6E2E6D2E702E2F16732E8F
:100CE000831203132F121230831203133202C03007
:100CF00003193102031C7D2E8F2E12303402C030B6
:100D000003193302031C8E2E852E1430340250300A
:100D10000319330203188E2E8D2E8F2E902E922EB5
:100D2000912E942EAF16972E83120313AF12143008
:100D3000831203133202503003193102031CA12E17
:100D4000B32E14303402503003193302031CB22E78
:100D5000A92E15303402E030031933020318B22EE5
:100D6000B12EB32EB42EB62EB52EB82E2F17BB2E05
:100D7000831203132F131530831203133202E03052
:100D800003193102031CC52ED72E15303402E03072
:100D900003193302031CD62ECD2E173034027030C7
:100DA000031933020318D62ED52ED72ED82EDA2EBD
:100DB000D92EDC2EAF17DF2E83120313AF1383124D
:100DC0000313A20A4B2CC028F601F401F5017208A6
:100DD0007304031DEE2EF001F10100341F30F60400
:100DE0000310F60AF20DF30D031CF12EF30CF20CB6
:100DF00073087102031DFE2E72087002031C062F79
:100E00007208F0027308031C730AF102F40DF50D69
:100E1000F60BF61AF62EF61F122FF409F40A031930
:100E2000F503F5097408F2007508F300761F003425
:100E3000F009F00A0319F103F10900348401831267
:100E40000313C801F31F332F0310FF30F007F0091D
:100E5000031CF107F109031CF207F209031CF30755
:100E6000F3094817C81777088039C806F71F4A2FB3
:100E70000310FF30F407F409031CF507F509031C00
:100E8000F607F609031CF707F7094A2F84018312B6
:100E90000313C801F801F901FA01FB017408750494
:100EA000760477040319572FC030C805622FF0016C
:100EB000F101F201F301F02F0310F40DF50DF60D21
:100EC000F70DC80AF71F5C2FC80A0310F80DF90DBB
:100ED000FA0DFB0D77087302031D782F7608720256
:100EE000031D782F75087102031D782F7408700296
:100EF000031C8A2F78147408F0027508031C750F00
:100F0000F1027608031C760FF2027708031C770FB4
:100F1000F3020310F70CF60CF50CF40CC8034808A8
:100F20003F39031D652F481FA22F0310FF30F00724
:100F3000F009031CF107F109031CF207F209031C75
:100F4000F307F3097008F4007108F5007208F60061
:100F50007308F7007808F0007908F1007A08F200C9
:100F60007B08F300C81FF02F0310FF30F007F009D3
:100F7000031CF107F109031CF207F209031CF30734
:100F8000F309F02F84017008F8007108F900720865
:100F9000FA007308FB00F201F301F001F101031004
:100FA000FB0CFA0CF90CF80C031CE42F7408F00786
:100FB00075080318750FF10776080318760FF20706
:100FC00077080318770FF307780879047A047B040D
:100FD0000319F02F0310F40DF50DF60DF70DCF2FBB
:100FE00084080319003473088000840372088000A9
:100FF000840371088000840370088000003430345A
:084000000000010000000000B7
:02400E00213F50
:00000001FF
